:020000040800F2
:1000000000060020E1010008E3010008E301000808
:10001000E3010008E3010008E3010008E301000830
:10002000E3010008E3010008E3010008CD35000802
:10003000E3010008E3010008E3010008E301000810
:10004000E3010008E3010008E3010008E301000800
:10005000E3010008E3010008753800089D38000836
:10006000C5380008ED38000815390008E30100081C
:10007000E3010008E3010008E3010008E3010008D0
:10008000E3010008E3010008E3010008E3010008C0
:10009000E3010008E3010008E30100083D3900081E
:1000A000E3010008E3010008E3010008E3010008A0
:1000B000253A0008E3010008E3010008E301000815
:1000C000E3010008E3010008E3010008E301000880
:1000D000E3010008113A0008E3010008E301000809
:1000E000A1390008E3010008E3010008E30100086A
:1000F000E3010008E3010008E3010008E301000850
:10010000E3010008E3010008E3010008E30100083F
:10011000E3010008E3010008E3010008E30100082F
:10012000E3010008E3010008E3010008E30100081F
:10013000E3010008E3010008E3010008E30100080F
:10014000E3010008E3010008E3010008812D000835
:10015000E3010008E3010008E3010008E3010008EF
:10016000E3010008E3010008E3010008E3010008DF
:10017000E3010008E3010008E3010008E3010008CF
:10018000E3010008E3010008E3010008E3010008BF
:10019000E3010008E3010008E3010008E3010008AF
:1001A000E3010008E3010008E3010008E30100089F
:1001B000E3010008E3010008E3010008E30100088F
:1001C000E3010008E3010008E3010008E30100087F
:1001D000E3010008E3010008E3010008E30100086F
:1001E00002E000F000F8FEE772B6374880F30888B6
:1001F000364880F3098836483649086040F20000E6
:10020000CCF200004EF63471CEF200010860BFF36C
:100210004F8FBFF36F8F40F20000C0F2F0004EF638
:100220008851CEF200010860BFF34F8FBFF36F8F8C
:100230004FF00000E1EE100A4EF63C71CEF20001E4
:100240000860062080F31488BFF36F8F02F060FA15
:1002500003F05AF94FF055301F491B4A91423CBFF9
:1002600041F8040BFAE71D49184A91423CBF41F896
:10027000040BFAE71A491B4A1B4B9A423EBF51F83E
:10028000040B42F8040BF8E700201849184A914281
:100290003CBF41F8040BFAE702F03EFA03F088F99C
:1002A000144C154DAC4203DA54F8041B8847F9E7A7
:1002B00000F042F8114C124DAC4203DA54F8041B22
:1002C0008847F9E702F026BA000600200022002045
:1002D0000000000808ED00E00000002000060020FB
:1002E000283E0008002200204C220020502200203E
:1002F000F0300020E0010008E0010008E001000803
:10030000E00100082DE9F04F2DED108AC1F80CD066
:10031000C3689D46BDEC108ABDE8F08F002383F3CF
:1003200011882846A047002001F0A6FDFEE701F055
:1003300035FD00DFFEE7000038B500F0D1FB02F02C
:10034000B7F9054602F0DAF90446C8B90E4B9D42EA
:1003500018D001339D4218BF044641F2883504BFCE
:1003600001240025002002F0ADF90CB100F074F872
:1003700000F02AFD284600F0BFF800F06DF8F9E71C
:100380000025EFE70546EDE7010007B008B500F0EE
:1003900073FBA0F120035842584108BD07B541F254
:1003A0001203022101A8ADF8043000F083FB03B072
:1003B0005DF804FB38B5302383F3118817480368D0
:1003C0000BB101F025FE164A144800234FF47A7150
:1003D00001F014FE002383F31188124C236813B13B
:1003E0002368013B2360636813B16368013B63606A
:1003F0000D4D2B7833B963687BB9022000F046FCC1
:10040000322363602B78032B07D163682BB902205A
:1004100000F03CFC4FF47A73636038BD502200203A
:10042000B50300087023002068220020084B1870D4
:1004300003280CD8DFE800F008050208022000F0CD
:1004400015BC022000F002BC024B00225A6070472B
:100450006822002070230020234B244A10B51C463C
:10046000196801313FD004339342F9D16268A24246
:1004700039D31F4B9B6803F1006303F540439A4255
:1004800031D2002000F046FB0220FFF7CFFF194BCE
:100490001A6C00221A64196E1A66196E596C5A6425
:1004A000596E5A665A6E5A6942F080025A615A6908
:1004B00022F080025A615A691A6942F000521A61A8
:1004C0001A6922F000521A611B6972B64FF0E023DC
:1004D0003021C3F8084DD4E9003281F311889D46DC
:1004E00083F30888104710BD00C0000820C0000832
:1004F00000220020003802402DE9F04F93B0AA4BB3
:1005000000902022FF210AA89D6800F007FCA74A5E
:100510001378A3B9A648012103601170302383F337
:10052000118803680BB101F073FDA24AA0480023B3
:100530004FF47A7101F062FD002383F31188009B70
:1005400013B19D4B009A1A609C4A009C1378032BB0
:100550001EBF00231370984A4FF0000A18BF536063
:10056000D3465646D146012000F080FB24B1924B81
:100570001B68002B00F01182002000F07DFA039030
:10058000039B002BF2DB012000F060FB039B213B6F
:10059000162BE8D801A252F823F000BFF905000895
:1005A00021060008B5060008670500086705000871
:1005B000670500083F0700080F0900082908000820
:1005C0008B080008B3080008D90800086705000870
:1005D000EB080008670500085D0900089906000897
:1005E00067050008A109000805060008990600082B
:1005F000670500088B0800080220FFF7C7FE0028E7
:1006000040F0F581009B0221BAF1000F08BF1C46A3
:1006100005A841F21233ADF8143000F04BFAA2E70E
:100620004FF47A7000F028FA071EEBDB0220FFF788
:10063000ADFE0028E6D0013F052F00F2DA81DFE8A9
:1006400007F0030A0D10133605230593042105A8AE
:1006500000F030FA17E054480421F9E75848042123
:10066000F6E758480421F3E74FF01C08404600F035
:1006700053FA08F104080590042105A800F01AFABD
:10068000B8F12C0FF2D1012000FA07F747EA0B0B63
:100690005FFA8BFB4FF0000900F08CFB26B10BF0EA
:1006A0000B030B2B08BF0024FFF778FE5BE74648DF
:1006B0000421CDE7002EA5D00BF00B030B2BA1D10D
:1006C0000220FFF763FE074600289BD0012000F0C0
:1006D00021FA0220FFF7AAFE00261FFA86F84046FC
:1006E00000F028FA044690B10021404600F032FAAA
:1006F00001360028F1D1BA46044641F21213022114
:1007000005A8ADF814303E4600F0D4F92BE70120DF
:10071000FFF78CFE2546244B9B68AB4207D9284641
:1007200000F0FAF9013040F067810435F3E7234B1C
:1007300000251D70204BBA465D603E46ACE7002E9A
:100740003FF460AF0BF00B030B2B7FF45BAF022089
:10075000FFF76CFE322000F08FF9B0F10008FFF6D1
:1007600051AF18F003077FF44DAF0F4A926808EBC2
:10077000050393423FF646AFB8F5807F3FF742AF9F
:10078000124B0193B84523DD4FF47A7000F074F9F1
:100790000390039A002AFFF635AF019B039A03F8F2
:1007A000012B0137EDE700BF002200206C23002061
:1007B00050220020B503000870230020682200208A
:1007C00004220020082200200C2200206C2200209D
:1007D000C820FFF7DBFD074600283FF413AF1F2DAD
:1007E00011D8C5F1200242450AAB25F0030028BF0D
:1007F000424683490192184400F06AFA019A8048FF
:10080000FF2100F08BFA4FEAA8037D490193C8F35A
:100810008702284600F08AFA064600283FF46DAFAA
:10082000019B05EB830537E70220FFF7AFFD0028AA
:100830003FF4E8AE00F0BAF900283FF4E3AE002739
:10084000B846704B9B68BB4218D91F2F11D80A9B22
:1008500001330ED027F0030312AA134453F8203CAF
:1008600005934046042205A900F00EFB043780469C
:10087000E7E7384600F050F90590F2E7CDF814802C
:10088000042105A800F016F906E70023642104A856
:10089000049300F005F900287FF4B4AE0220FFF7BE
:1008A00075FD00283FF4AEAE049800F067F905909E
:1008B000E6E70023642104A8049300F0F1F800287F
:1008C0007FF4A0AE0220FFF761FD00283FF49AAE4E
:1008D000049800F063F9EAE70220FFF757FD0028CB
:1008E0003FF490AE00F072F9E1E70220FFF74EFD11
:1008F00000283FF487AE05A9142000F06DF904210B
:100900000746049004A800F0D5F83946B9E732202C
:1009100000F0B2F8071EFFF675AEBB077FF472AEAB
:10092000384A926807EB090393423FF66BAE022008
:10093000FFF72CFD00283FF465AE27F003074F4476
:10094000B9453FF4A9AE484600F0E6F80421059009
:1009500005A800F0AFF809F10409F1E74FF47A7047
:10096000FFF714FD00283FF44DAE00F01FF90028FA
:1009700044D00A9B01330BD008220AA9002000F0C2
:10098000D5F900283AD02022FF210AA800F0C6F9A4
:10099000FFF704FD1C4801F075FA13B0BDE8F08FB5
:1009A000002E3FF42FAE0BF00B030B2B7FF42AAE7F
:1009B0000023642105A8059300F072F8074600287B
:1009C0007FF420AE0220FFF7E1FC804600283FF4D0
:1009D00019AEFFF7E3FC41F2883001F053FA0598B5
:1009E00000F030FA464600F0E5F93C46BBE5064625
:1009F00052E64FF0000905E6BA467EE637467CE649
:100A00006C22002000220020A08601002DE9F84F72
:100A10004FF47A73DFF85880DFF8589006460D4699
:100A200002FB03F7002498F900305A1C5FFA84FA9D
:100A300001D0A34212D159F8240003682A46D3F802
:100A400020B031463B46D847854207D1074B0120AD
:100A500083F800A0BDE8F88F0124E4E7002CFBD068
:100A60004FF4FA7001F00EFA0020F3E7B8230020EB
:100A7000102200201422002007B500230246012185
:100A80000DF107008DF80730FFF7C0FF20B19DF88A
:100A9000070003B05DF804FB4FF0FF30F9E70000FA
:100AA0000A4608B50421FFF7B1FF80F00100C0B28B
:100AB000404208BD30B4074B0A461978064B53F83C
:100AC00021402368DD69054B0146AC46204630BC19
:100AD000604700BFB823002014220020A086010038
:100AE00070B501F0EBFC094E094D308000242868F8
:100AF0003388834208D901F0DBFC2B6804440133BE
:100B0000B4F5404F2B60F2D370BD00BFBA23002074
:100B10007823002001F080BD00F1006000F5404026
:100B20000068704700F10060920000F5404001F05D
:100B30000BBD0000054B1A68054B1B889B1A8342AE
:100B400002D9104401F0B4BC002070477823002083
:100B5000BA23002038B5084D044629B1286820443E
:100B6000BDE8384001F0C4BC2868204401F0A8FC6E
:100B70000028F3D038BD00BF7823002010F0030315
:100B80000AD1B0F5047F05D200F10050A0F5104065
:100B9000D0F80038184670470023FBE700F10050FA
:100BA000A0F51040D0F8100A70470000064991F8EF
:100BB000243033B10023086A81F824300822FFF77B
:100BC000B1BF0120704700BF7C230020014B186893
:100BD000704700BF002004E070B5194B1D68194B29
:100BE0000138C5F30B0408442D0C04221E88A642CC
:100BF0000BD15C680A46013C824213460FD214F9BD
:100C0000016F4EB102F8016BF6E7013A03F10803F8
:100C1000ECD181420B4602D22C2203F8012B0A4A66
:100C200005241688AE4204D1984284BF967803F812
:100C3000016B013C02F10402F3D1581A70BD00BFF0
:100C4000002004E0143B0008003B0008022804D107
:100C5000054B4FF080429A6170470128FCD1024B4E
:100C60004FF00052F7E700BF00000240022804D115
:100C7000054B4FF480429A6170470128FCD1024B2A
:100C80004FF40052F7E700BF00000240022805D1F0
:100C9000064A536983F48043536170470128FCD1AD
:100CA000024A536983F40053F6E700BF0000024094
:100CB00070B504464FF47A764CB1412C254628BFD6
:100CC000412506FB05F001F0DDF8641BF4E770BD7B
:100CD00010B50023934203D0CC5CC4540133F9E730
:100CE00010BD000010B5013810F9013F3BB191F97A
:100CF00000409C4203D11AB10131013AF4E71AB124
:100D000091F90020981A10BD1046FCE703460246F0
:100D1000D01A12F9011B0029FAD170470244034688
:100D2000934202D003F8011BFAE770472DE9F8431C
:100D30001F4D144695F824200746884652BBDFF81D
:100D400070909CB395F824302BB92022FF2148469F
:100D50002F62FFF7E3FF95F82400C0F10802A242DA
:100D600028BF2246D6B24146920005EB8000FFF72D
:100D7000AFFF95F82430A41B1E44F6B2082E17448A
:100D80009044E4B285F82460DBD1FFF70FFF002820
:100D9000D7D108E02B6A03EB82038342CFD0FFF761
:100DA00005FF0028CBD10020BDE8F8830120FBE738
:100DB0007C230020024B1A78024B1A70704700BF48
:100DC000B82300201022002038B5194C194D2046B8
:100DD00000F0BEFB2946204600F0E6FB2D686A6D58
:100DE000D2F8043843F00203C2F804384FF47A70A2
:100DF000FFF75EFF1049284600F0DCFC6A6D0F4DDE
:100E0000D2F8043828680E4923F00203C2F80438E7
:100E1000A0424FF4E1330B6001D000F0F9FA6868AA
:100E2000A04204D0BDE83840054900F0F1BA38BD11
:100E300098280020183C0008203C000814220020BC
:100E4000A423002070B50C4B0C4D1E780C4B55F8AC
:100E500026209A4204460DD00A4B0021142218463F
:100E6000FFF75CFF0460014655F82600BDE87040BE
:100E700000F0CEBA70BD00BFB823002014220020BD
:100E800098280020A423002030B5094D0A4491423F
:100E90000DD011F8013B5840082340F30004013BFA
:100EA0002C4013F0FF0384EA5000F6D1EFE730BD89
:100EB0002083B8ED026843681143016003B118470D
:100EC00070470000024AD36843F0C003D360704704
:100ED0000010014010B5084C084A0021204600F0DF
:100EE00075FA074BC4F85C3203F1454303F52D4313
:100EF000C4F8603210BD00BFBC230020C50E00083E
:100F000000100140234A037C002918BF0A46012B28
:100F100030B5C0F868220CD11F4B984209D11F4B45
:100F2000596C41F010015964596E41F01001596635
:100F30005B6EB2F904501468D0F86032D0F85C12DD
:100F4000002D03EB5403B3FBF4F3BEBF23F00705FE
:100F500003F0070343EA450394888B60D38843F08A
:100F600040030B61138943F001034B6144F40453C4
:100F700043F02C03CB6004F4A05400230B60B4F5C1
:100F8000806F0B684B680CBF7F23FF2380F86432AF
:100F900030BD00BF343B0008BC23002000380240B5
:100FA0002DE9F041D0F85C62F7683368DA05044651
:100FB0009DB20DD5302383F311884FF48061043046
:100FC000FFF778FF6FF480733360002383F3118899
:100FD000302383F3118804F1040815F02F033AD16C
:100FE00083F31188380615D5290613D5302383F3EA
:100FF000118804F1380000F065F900284EDA082164
:10100000201DFFF757FF4FF67F733B40F36000232F
:1010100083F311887A0616D56B0614D5302383F333
:101020001188D4E913239A420AD1236C43B127F0E3
:1010300040073F041021201D3F0CFFF73BFFF760E6
:10104000002383F31188D4F86822D36843B3BDE842
:10105000F041106918472B0714D015F0080F0CBF8A
:1010600000214FF48071E80748BF41F02001AA0732
:1010700048BF41F040016B0748BF41F08001404646
:10108000FFF718FFAD06736805D594F86412204683
:10109000194000F0CBF93568ADB29EE77060B6E755
:1010A000BDE8F081F8B5154682680669AA420B468C
:1010B000816938BF8568761AB54204460BD2184656
:1010C0002A46FFF705FEA3692B44A361A3685B1BB7
:1010D000A3602846F8BD0CD918463246FFF7F8FD44
:1010E000AF1BE1683A463044FFF7F2FDE3683B444A
:1010F000EBE718462A46FFF7EBFDE368E5E700005B
:1011000083689342F7B51546044638BF8568D0E931
:101110000460361AB5420BD22A46FFF7D9FD63693F
:101120002B446361A36828465B1BA36003B0F0BD3A
:101130000DD932460191FFF7CBFD0199E068AF1B55
:101140003A463144FFF7C4FDE3683B44E9E72A46E9
:10115000FFF7BEFDE368E4E710B50A440024C3616D
:10116000029B8460C0E90000C0E90511C160026112
:10117000036210BD08B5D0E90532934201D18268FF
:1011800082B98268013282605A1C42611970D0E9CA
:1011900004329A4224BFC3684361002100F08EFEEE
:1011A000002008BD4FF0FF30FBE7000070B5302392
:1011B00004460E4683F31188A568A5B1A368A26909
:1011C000013BA360531CA36115782269934224BF9D
:1011D000E368A361E3690BB120469847002383F3DA
:1011E0001188284607E03146204600F057FE0028C7
:1011F000E2DA85F3118870BD2DE9F74F04460E46FB
:1012000017469846D0F81C904FF0300A8AF31188A0
:101210004FF0000B154665B12A4631462046FFF7D0
:1012200041FF034660B94146204600F037FE0028E2
:10123000F1D0002383F31188781B03B0BDE8F08F51
:10124000B9F1000F03D001902046C847019B8BF3F2
:101250001188ED1A1E448AF31188DCE7C0E90511F4
:10126000C160C3611144009B8260C0E9000001615C
:1012700003627047F8B504460D461646302383F3E3
:101280001188A768A7B1A368013BA36063695A1CD2
:1012900062611D70D4E904329A4224BFE36863613D
:1012A000E3690BB120469847002080F3118807E0DE
:1012B0003146204600F0F2FD0028E2DA87F311887B
:1012C000F8BD0000D0E905239A4210B501D182682B
:1012D0007AB98268013282605A1C82611C78036983
:1012E0009A4224BFC3688361002100F0E7FD2046D5
:1012F00010BD4FF0FF30FBE72DE9F74F04460E46D7
:1013000017469846D0F81C904FF0300A8AF311889F
:101310004FF0000B154665B12A4631462046FFF7CF
:10132000EFFE034660B94146204600F0B7FD0028B5
:10133000F1D0002383F31188781B03B0BDE8F08F50
:10134000B9F1000F03D001902046C847019B8BF3F1
:101350001188ED1A1E448AF31188DCE7026843689D
:101360001143016003B11847704700001430FFF7C4
:1013700043BF00004FF0FF331430FFF73DBF0000C4
:101380003830FFF7B9BF00004FF0FF333830FFF7B8
:10139000B3BF00001430FFF709BF00004FF0FF316A
:1013A0001430FFF703BF00003830FFF763BF0000C1
:1013B0004FF0FF323830FFF75DBF0000012914BF46
:1013C0006FF0130000207047FFF784BD37B5154656
:1013D0000E4A026000224260C0E902220122044655
:1013E00002740B46009000F15C014FF480721430DF
:1013F000FFF7B2FE00942B464FF4807204F5AE71F5
:1014000004F13800FFF72AFF03B030BD483B000865
:1014100010B53023044683F31188FFF773FD0223D0
:101420002374002080F3118810BD000038B5C36913
:1014300004460D461BB904210844FFF78FFF2946D7
:1014400004F11400FFF796FE002806DA201D4FF481
:101450000061BDE83840FFF781BF38BD02684368CE
:101460001143016003B118477047000013B5446B86
:10147000D4F894341A681178042915D1217C0229F2
:1014800012D11979128901238B4013420CD101A981
:1014900004F14C0001F0F4FED4F89444019B21794E
:1014A0000246206800F0D0F902B010BD143001F0FF
:1014B00077BE00004FF0FF33143001F071BE000022
:1014C0004C3001F049BF00004FF0FF334C3001F0C9
:1014D00043BF0000143001F045BE00004FF0FF3163
:1014E000143001F03FBE00004C3001F015BF000089
:1014F0004FF0FF324C3001F00FBF0000002070476A
:1015000010B5D0F894341A6811780429044617D11C
:10151000017C022914D15979528901238B4013424D
:101520000ED1143001F0D8FD024648B1D4F89444ED
:101530004FF4807361792068BDE8104000F072B903
:1015400010BD0000406BFFF7DBBF000070470000DC
:101550007FB5124B036000234360C0E902330125CD
:1015600002260F4B057404460290019300F1840299
:10157000294600964FF48073143001F089FD094B21
:101580000294CDE9006304F523724FF48073294679
:1015900004F14C0001F050FE04B070BD703B000837
:1015A000451500086D1400080B68302282F311887D
:1015B0000A7903EB820290614A79093243F82200EA
:1015C0008A7912B103EB820398610223C0F8941464
:1015D0000374002080F311887047000038B5037F42
:1015E000044613B190F85430ABB9201D01250221F7
:1015F000FFF734FF04F1140025776FF0010100F0CC
:1016000069FC84F8545004F14C006FF00101BDE80E
:10161000384000F05FBC38BD10B5012104460430ED
:10162000FFF71CFF0023237784F8543010BD00001F
:1016300038B504460025143001F042FD04F14C0099
:10164000257701F011FE201D84F854500121FFF789
:1016500005FF2046BDE83840FFF752BF90F8443000
:1016600003F06003202B07D190F84520212A4FF08A
:10167000000303D81F2A06D800207047222AFBD176
:10168000C0E90E3303E0034A82630722C2630364A6
:10169000012070471C22002037B5D0F894341A6816
:1016A0001178042904461AD1017C022917D119792D
:1016B000128901238B40134211D100F14C052846B9
:1016C00001F092FE58B101A9284601F0D9FDD4F8E5
:1016D0009444019B21790246206800F0B5F803B0DC
:1016E00030BD0000F0B500EB810385B09E69044673
:1016F0000D46FEB1302383F3118804EB8507301DBE
:101700000821FFF7ABFEFB685B691B6806F14C0024
:101710001BB1019001F0C2FD019803A901F0B0FDD9
:10172000024648B1039B2946204600F08DF800236D
:1017300083F3118805B0F0BDFB685A691268002A6E
:10174000F5D01B8A013B1340F1D104F14402EAE7D2
:10175000093138B550F82140DCB1302383F31188CA
:10176000D4F894241368527903EB8203DB689B69F5
:101770005D6845B104216018FFF770FE294604F149
:10178000140001F0B3FC2046FFF7BAFE002383F3F8
:10179000118838BD7047000001F012B801230370B2
:1017A0000023C0E90133C36183620362C362436201
:1017B0000363704738B50446302383F3118800254E
:1017C000C0E90355C0E90555416001F009F802235D
:1017D000237085F31188284638BD000070B500EBF2
:1017E000810305465069DA600E46144618B110228E
:1017F0000021FFF793FAA06918B110220021FFF72A
:101800008DFA31462846BDE8704001F0B3B80000BB
:10181000826802F0011282600022C0E90422826123
:1018200001F034B9F0B400EB81044789E468012584
:10183000A4698D403D43458123600023A26063601D
:10184000F0BC01F04FB90000F0B400EB810407894F
:10185000E468012564698D403D43058123600023D0
:10186000A2606360F0BC01F0C9B9000070B502234A
:10187000002504460370C0E90255C0E90455C5645B
:10188000856180F8345001F011F863681B6823B15A
:1018900029462046BDE87040184770BD0378052BE7
:1018A00010B504460AD080F8503005230370436811
:1018B0001B680BB1042198470023A36010BD0000F2
:1018C0000178052906D190F85020436802701B6802
:1018D00003B118477047000070B590F834300446E3
:1018E00013B1002380F8343004F14402204601F0A3
:1018F000EFF863689B68B3B994F8443013F060055F
:1019000035D00021204601F08FFB0021204601F058
:1019100081FB63681B6813B10621204698470623A4
:1019200084F8343070BD204698470028E4D0B4F8DD
:101930004A30E26B9A4288BFE36394F94430E56B26
:10194000002B4FF0300380F20381002D00F0F28075
:10195000092284F8342083F311880021D4E90E236E
:101960002046FFF771FF002383F31188DAE794F82C
:10197000452003F07F0343EA022340F20232934200
:1019800000F0C58021D8B3F5807F48D00DD8012B59
:101990003FD0022B00F09380002BB2D104F14C0217
:1019A000A2630222E2632364C1E7B3F5817F00F002
:1019B0009B80B3F5407FA4D194F84630012BA0D191
:1019C000B4F84C3043F0020332E0B3F5006F4DD071
:1019D00017D8B3F5A06F31D0A3F5C063012B90D811
:1019E000636894F846205E6894F84710B4F848306D
:1019F0002046B047002884D04368A3630368E363AC
:101A00001AE0B3F5106F36D040F6024293427FF4ED
:101A100078AF5C4BA3630223E3630023C3E794F82E
:101A20004630012B7FF46DAFB4F84C3023F0020345
:101A3000C4E90E55A4F84C30256478E7B4F8443076
:101A4000B3F5A06F0ED194F8463084F84E3020469E
:101A500000F084FF63681B6813B10121204698479A
:101A6000032323700023C4E90E339CE704F14F03E2
:101A7000A3630123C3E72378042B10D1302383F31E
:101A800011882046FFF7C4FE85F31188032163689F
:101A900084F84F5021701B680BB12046984794F88A
:101AA0004630002BDED084F84F3004232370636867
:101AB0001B68002BD6D0022120469847D2E794F825
:101AC00048301D0603F00F0120460AD500F0F2FF52
:101AD000012804D002287FF414AF2B4B9AE72B4B3C
:101AE00098E700F0D9FFF3E794F84630002B7FF435
:101AF00008AF94F8483013F00F01B3D01A0620460F
:101B000002D501F0A5FAADE701F098FAAAE794F83A
:101B10004630002B7FF4F5AE94F8483013F00F01F7
:101B2000A0D01B06204602D501F07EFA9AE701F00C
:101B300071FA97E7142284F8342083F311882B4636
:101B40002A4629462046FFF76DFE85F31188E9E60F
:101B50005DB1152284F8342083F311880021D4E983
:101B60000E232046FFF75EFEFDE60B2284F83420AC
:101B700083F311882B462A4629462046FFF764FE48
:101B8000E3E700BFA03B0008983B00089C3B00082F
:101B900038B590F834300446002B3ED0063BDAB21C
:101BA0000F2A34D80F2B32D8DFE803F03731310851
:101BB000223231313131313131313737C56BB0F803
:101BC0004A309D4214D2C3681B8AB5FBF3F203FB73
:101BD00012556DB9302383F311882B462A462946C6
:101BE000FFF732FE85F311880A2384F834300EE0C3
:101BF000142384F83430302383F3118800231A46E9
:101C000019462046FFF70EFE002383F3118838BDE6
:101C1000036C03B198470023E7E70021204601F059
:101C200003FA0021204601F0F5F963681B6813B13F
:101C30000621204698470623D7E7000010B590F804
:101C40003430142B044629D017D8062B05D001D8E0
:101C50001BB110BD093B022BFBD80021204601F02F
:101C6000E3F90021204601F0D5F963681B6813B140
:101C7000062120469847062319E0152BE9D10B23AE
:101C800080F83430302383F3118800231A46194634
:101C9000FFF7DAFD002383F31188DAE7C3689B6955
:101CA0005B68002BD5D1036C03B19847002384F8FF
:101CB0003430CEE700230375826803691B68996896
:101CC0009142FBD25A6803604260106058607047CE
:101CD00000230375826803691B6899689142FBD8E9
:101CE0005A680360426010605860704708B5084643
:101CF000302383F311880B7D032B05D0042B0DD0EB
:101D00002BB983F3118808BD8B6900221A604FF04C
:101D1000FF338361FFF7CEFF0023F2E7D1E9003202
:101D200013605A60F3E70000FFF7C4BF054BD968A2
:101D30000875186802681A60536001220275D8603D
:101D4000FEF7E0BA2826002030B50C4BDD684B1CAE
:101D500087B004460FD02B46094A684600F04EF97A
:101D60002046FFF7E3FF009B13B1684600F050F9EF
:101D7000A86907B030BDFFF7D9FFF9E72826002092
:101D8000ED1C0008044B1A68DB6890689B68984259
:101D900094BF00200120704728260020084B10B572
:101DA0001C68D86822681A60536001222275DC60C2
:101DB000FFF78EFF01462046BDE81040FEF7A2BAAD
:101DC0002826002038B5074C07490848012300257C
:101DD0002370656001F040FB0223237085F31188B6
:101DE00038BD00BF90280020A83B0008282600200E
:101DF00000F044B9034A516853685B1A9842FBD813
:101E0000704700BF001000E08B60022308618B82E6
:101E1000084670478368A3F1840243F8142C0269D2
:101E200043F8442C426943F8402C094A43F8242CD7
:101E3000C26843F8182C022203F80C2C002203F885
:101E40000B2C044A43F8102CA3F12000704700BF6C
:101E50001D0300082826002008B5FFF7DBFFBDE8BA
:101E60000840FFF761BF0000024BDB6898610F205C
:101E7000FFF75CBF28260020302383F31188FFF78B
:101E8000F3BF000008B50146302383F31188082012
:101E9000FFF75AFF002383F3118808BD064BDB6868
:101EA00039B1426818605A60136043600420FFF73C
:101EB0004BBF4FF0FF307047282600200368984240
:101EC00006D01A680260506099611846FFF72CBF6F
:101ED0007047000038B504460D462068844200D1A2
:101EE00038BD036823605C608561FFF71DFFF4E780
:101EF00010B503689C68A2420CD85C688A600B60CD
:101F00004C602160596099688A1A9A604FF0FF33DB
:101F1000836010BD1B68121BECE700000A2938BF64
:101F20000A2170B504460D460A26601901F08EFAA2
:101F300001F07AFA041BA54203D8751C2E4604460C
:101F4000F3E70A2E04D9BDE87040012001F0C4BABD
:101F500070BD0000F8B5144B0D46D96103F11001B6
:101F600041600A2A1969826038BF0A22016048600C
:101F70001861A818144601F05BFA0A2701F054FA18
:101F8000431BA342064606D37C1C281901F05EFAC7
:101F900027463546F2E70A2F04D9BDE8F84001206C
:101FA00001F09ABAF8BD00BF28260020F8B5064611
:101FB0000D4601F039FA0F4A134653F8107F9F423D
:101FC00006D12A4601463046BDE8F840FFF7C2BFB9
:101FD000D169BB68441A2C1928BF2C46A34202D9E8
:101FE0002946FFF79BFF224631460348BDE8F840EB
:101FF000FFF77EBF282600203826002010B4C0E955
:10200000032300235DF8044B4361FFF7CFBF0000BB
:1020100010B5194C236998420DD0D0E9003281687F
:1020200013605A609A680A449A60002303604FF074
:10203000FF33A36110BD2346026843F8102F53609D
:102040000022026022699A4203D1BDE8104001F0EB
:10205000F7B9936881680B44936001F0E5F9226950
:10206000E1699268441AA242E4D91144BDE81040E3
:10207000091AFFF753BF00BF282600202DE9F047BB
:10208000DFF8BC8008F110072C4ED8F8105001F092
:10209000CBF9D8F81C40AA68031B9A423ED81444D6
:1020A000D5E900324FF00009C8F81C4013605A60AF
:1020B000C5F80090D8F81030B34201D101F0C0F952
:1020C00089F31188D5E9033128469847302383F3F3
:1020D00011886B69002BD8D001F0A6F96A69A0EBD2
:1020E00004094A4582460DD2022001F0F5F900228A
:1020F000D8F81030B34208D151462846BDE8F04721
:10210000FFF728BF121A2244F2E712EB090938BF81
:102110004A4629463846FFF7EBFEB5E7D8F81030B7
:10212000B34208D01444211AC8F81C00A960BDE8C5
:10213000F047FFF7F3BEBDE8F08700BF3826002068
:102140002826002000207047FEE7000070470000AE
:102150004FF0FF307047000002290CD0032904D053
:102160000129074818BF00207047032A05D80548F1
:1021700000EBC2007047044870470020704700BF62
:102180007C3C00082C220020303C000870B59AB03E
:102190000546084601A9144600F0C2F801A8FEF75A
:1021A000B5FD431C5B00C5E9003400222370032306
:1021B0006370C6B201AB02341046D1B28E4204F154
:1021C000020401D81AB070BD13F8011B04F8021CF8
:1021D00004F8010C0132F0E708B5302383F31188CD
:1021E0000348FFF759FA002383F3118808BD00BFA5
:1021F0009828002090F8443003F01F02012A07D1EC
:1022000090F845200B2A03D10023C0E90E3315E0D6
:1022100003F06003202B08D1B0F848302BB990F8B8
:102220004520212A03D81F2A04D8FFF717BA222AEB
:10223000EBD0FAE7034A82630722C26303640120FA
:10224000704700BF2322002007B5052917D8DFE813
:1022500001F0191603191920302383F31188104A4D
:1022600001900121FFF7BAFA01980E4A0221FFF707
:10227000B5FA0D48FFF7DCF9002383F3118803B0AA
:102280005DF804FB302383F311880748FFF7A6F9B4
:10229000F2E7302383F311880348FFF7BDF9EBE73A
:1022A000D03B0008F43B00089828002038B50C4DBE
:1022B0000C4C0D492A4604F10800FFF767FF05F1B1
:1022C000CA0204F110000949FFF760FF05F5CA7260
:1022D00004F118000649BDE83840FFF757BF00BFBA
:1022E000602D00202C220020B43B0008B93B0008E0
:1022F000C43B000870B5044608460D46FEF706FDCF
:10230000C6B22046013403780BB9184670BD324678
:102310002946FEF7E7FC0028F3D10120F6E700008C
:102320002DE9F84F05460C46FEF7F0FC2949C6B2E8
:102330002846FFF7DFFF28492846FFF7DBFF08B1F3
:102340001036F6B2632E0DD8DFF88880DFF888905B
:10235000224FDFF890A0DFF890B02E7846B92670B3
:10236000BDE8F88F29462046BDE8F84F01F0AABB2A
:10237000252E2BD1072241462846FEF7B3FC58B93B
:10238000DBF800302360BBF80430A3809BF80630F4
:10239000A37107350734E0E7082249462846FEF7CF
:1023A000A1FC98B90E4BA21C197809090232C95D2B
:1023B00002F8041C13F8011B01F00F015345C95D1D
:1023C00002F8031CF0D118340835C6E704F8016B95
:1023D0000135C2E79C3C0008C43B0008AC3C000847
:1023E000107AFF1F1C7AFF1FA43C0008BFF34F8F19
:1023F000024AD368DB03FCD4704700BF003C0240B4
:1024000008B5094B1B7873B9FFF7F0FF074B1A6942
:10241000002ABFBF064A5A6002F188325A601A6821
:1024200022F480621A6008BDBE2F0020003C0240EA
:102430002301674508B50B4B1B7893B9FFF7D6FF0F
:10244000094B1A6942F000421A611A6842F480523C
:102450001A601A6822F480521A601A6842F4806284
:102460001A6008BDBE2F0020003C02400B28F0B5CA
:1024700016D80C4C0C4923787BB90C4D0E460C2316
:102480004FF0006255F8047B46F8042B013B13F033
:10249000FF033A44F6D10123237051F82000F0BD28
:1024A0000020FCE7F02F0020C02F0020C03C0008D7
:1024B000014B53F820007047C03C00080C207047C7
:1024C0000B2810B5044601D9002010BDFFF7CEFF40
:1024D000064B53F824301844C21A0BB90120F4E714
:1024E00012680132F0D1043BF6E700BFC03C00089F
:1024F0000B2810B5044621D8FFF778FFFFF780FFBF
:102500000F4AF323D360C300DBB243F4007343F0FC
:1025100002031361136943F480331361FFF766FF0D
:10252000FFF7A4FF074B53F8241000F0D9F8FFF78A
:1025300081FF2046BDE81040FFF7C2BF002010BD5C
:10254000003C0240C03C0008F8B512F001031446FC
:1025500042D18218B2F1016F57D82D4B1B6813F08E
:10256000010352D02B4DFFF74BFFF323EB60FFF736
:102570003DFF40F20127032C15D824F00104661812
:10258000244C401A40F20117B142236900EB0105C7
:1025900024D123F001032361FFF74CFF0120F8BD94
:1025A000043C0430E7E78307E7D12B6923F4407349
:1025B0002B612B693B432B6151F8046B0660BFF321
:1025C0004F8FFFF713FF03689E42E9D02B6923F07A
:1025D00001032B61FFF72EFF0020E0E723F4407397
:1025E000236123693B4323610B882B80BFF34F8F0B
:1025F000FFF7FCFE2D8831F8023BADB2AB42C3D0F1
:10260000236923F001032361E4E71846C7E700BF0D
:1026100000380240003C0240084908B50B7828B158
:102620001BB9FFF7EDFE01230B7008BD002BFCD09A
:10263000BDE808400870FFF7FDBE00BFBE2F0020B8
:1026400010B50244064BD2B2904200D110BD441CDA
:1026500000B253F8200041F8040BE0B2F4E700BFE9
:10266000502800400F4B30B51C6F240407D41C6F5A
:1026700044F400741C671C6F44F400441C670A4C4B
:10268000236843F4807323600244084BD2B2904223
:1026900000D130BD441C00B251F8045B43F8205017
:1026A000E0B2F4E7003802400070004050280040DB
:1026B00007B5012201A90020FFF7C2FF019803B06E
:1026C0005DF804FB13B50446FFF7F2FFA04205D006
:1026D000012201A900200194FFF7C4FF02B010BD40
:1026E00070470000034B1A681AB9034AD2F87428DD
:1026F0001A607047F42F00200030024008B5FFF741
:10270000F1FF024B1868C0F3407008BDF42F0020A1
:1027100070470000FEE700000A4B0B480B4A90424E
:102720000BD30B4BDA1C121AC11E22F003028B4290
:1027300038BF00220021FEF7F1BA53F8041B40F81D
:10274000041BECE7743E0008F0300020F03000205D
:10275000F030002070B5D0E915439E6800224FF09C
:10276000FF3504EB42135101D3F800090028BEBF26
:10277000D3F8000940F08040C3F80009D3F8000BFB
:102780000028BEBFD3F8000B40F08040C3F8000B18
:10279000013263189642C3F80859C3F8085BE0D2C7
:1027A0004FF00113C4F81C3870BD0000890141F0DE
:1027B0002001016103699B06FCD41220FFF71ABBBC
:1027C00010B5054C2046FEF7E9FF4FF0A0436365C6
:1027D000024BA36510BD00BFF82F0020143D000878
:1027E00070B50378012B054650D12A4B446D9842B1
:1027F0001BD1294B5A6B42F080025A635A6D42F04A
:1028000080025A655A6D5A6942F080025A615A69CB
:1028100022F080025A610E2143205B6900F022FC05
:102820001E4BE3601E4BC4F800380023C4F8003E82
:10283000C02323606E6D4FF40413A3633369002B30
:10284000FCDA012333610C20FFF7D4FA3369DB078C
:10285000FCD41220FFF7CEFA3369002BFCDA0026F5
:10286000A6602846FFF776FF6B68C4F81068DB683F
:10287000C4F81468C4F81C684BB90A4BA3614FF044
:10288000FF336361A36843F00103A36070BD064B8F
:10289000F4E700BFF82F0020003802404014004049
:1028A00003002002003C30C0083C30C0F8B5446D45
:1028B000054600212046FFF779FFA96D00234FF060
:1028C00001128F68C4F834384FF00066C4F81C2831
:1028D0004FF0FF3004EB431201339F42C2F800690E
:1028E000C2F8006BC2F80809C2F8080BF2D20B68F4
:1028F0006A6DEB65636210231361166916F01006AA
:10290000FBD11220FFF776FAD4F8003823F4FE63E7
:10291000C4F80038A36943F4402343F01003A361D3
:102920000923C4F81038C4F814380A4BEB604FF090
:10293000C043C4F8103B084BC4F8003BC4F810690E
:10294000C4F80039EB6D03F1100243F48013EA651B
:10295000A362F8BDF03C000840800010426D90F882
:102960004E10D2F8003823F4FE6343EA0113C2F894
:10297000003870472DE9F84300EB8103456DDA68B4
:10298000166806F00306731E022B05EB41130C4676
:1029900080460FFA81F94FEA41104FF00001C3F869
:1029A000101B4FF0010104F1100398BFB60401FAA7
:1029B00003F391698EBF334E06F1805606F500464B
:1029C00000293AD0578A04F15801490137436F5022
:1029D000D5F81C180B43C5F81C382B180021C3F878
:1029E000101953690127611EA7409BB3138A928B6C
:1029F0009B08012A88BF5343D8F85C20981842EA04
:102A0000034301F1400205EB8202C8F85C00214655
:102A100053602846FFF7CAFE08EB8900C3681B8A8B
:102A200043EA8453483464011E432E51D5F81C38C0
:102A30001F43C5F81C78BDE8F88305EB4917D7F8A4
:102A4000001B21F40041C7F8001BD5F81C1821EA2F
:102A50000303C0E704F13F0305EB83030A4A5A600E
:102A600028462146FFF7A2FE05EB4910D0F80039B1
:102A700023F40043C0F80039D5F81C3823EA0707CF
:102A8000D7E700BF0080001000040002826D1268CA
:102A9000C265FFF75FBE00005831436D49015B58C6
:102AA00013F4004004D013F4001F0CBF02200120D7
:102AB000704700004831436D49015B5813F40040F2
:102AC00004D013F4001F0CBF022001207047000047
:102AD00000EB8101CB68196A0B6813604B68536087
:102AE0007047000000EB810330B5DD68AA69136808
:102AF000D36019B9402B84BF402313606B8A1468DC
:102B0000426D1C44013CB4FBF3F46343033323F0F4
:102B1000030302EB411043EAC44343F0C043C0F84F
:102B2000103B2B6803F00303012B09B20ED1D2F83E
:102B3000083802EB411013F4807FD0F8003B14BF3B
:102B400043F0805343F00053C0F8003B02EB4112C6
:102B5000D2F8003B43F00443C2F8003B30BD000014
:102B60002DE9F041244D6E6D06EB40130446D3F879
:102B7000087BC3F8087B38070AD5D6F8143819073C
:102B800006D505EB84032146DB6828465B68984739
:102B9000FA071FD5D6F81438DB071BD505EB8403DD
:102BA000D968CCB98B69488A5A68B2FBF0F600FB49
:102BB00016228AB91868DA6890420DD2121AC3E94F
:102BC0000024302383F311880B482146FFF78AFF46
:102BD00084F31188BDE8F081012303FA04F26B89C4
:102BE00023EA02036B81CB68002BF3D02146024815
:102BF000BDE8F041184700BFF82F002000EB81032B
:102C000070B5DD68436D6C692668E6604A0156BBA5
:102C10001A444FF40020C2F810092A6802F0030297
:102C2000012A0AB20ED1D3F8080803EB421410F4BB
:102C3000807FD4F8000914BF40F0805040F000506D
:102C4000C4F8000903EB4212D2F8000940F0044036
:102C5000C2F80009D3F83408012202FA01F1014355
:102C6000C3F8341870BD19B9402E84BF40202060CD
:102C700020682E8A8419013CB4FBF6F440EAC44073
:102C800040F000501A44C6E72DE9F8433B4D6E6D05
:102C900006EB40130446D3F80889C3F8088918F0F6
:102CA000010F4FEA40171AD0D6F81038DB0716D5B7
:102CB00005EB8003D9684B691868DA68904230D216
:102CC000121A4FF000091A60C3F80490302383F3FE
:102CD000118821462846FFF791FF89F3118818F0E3
:102CE000800F1CD0D6F834380126A640334216D0C7
:102CF00005EB84036D6DD3F80CC0DCF814200134AF
:102D0000E4B2D2F800E005EB04342F445168714579
:102D100015D3D5F8343823EA0606C5F83468BDE87B
:102D2000F883012303FA04F22B8923EA02032B819F
:102D30008B68002BD3D0214628469847CFE7BCF8B4
:102D40001000AEEB0103834228BF0346D7F81809F1
:102D500080B2B3EB800FE2D89068A0F1040959F873
:102D6000048FC4F80080A0EB09089844B8F1040F60
:102D7000F5D818440B4490605360C7E7F82F002043
:102D80002DE9F74FA24C656D6E69AB691E4016F4D4
:102D900080586E6107D02046FEF768FD03B0BDE89D
:102DA000F04F00F047BC002E12DAD5F8003E9848EC
:102DB0009B071EBFD5F8003E23F00303C5F8003E75
:102DC000D5F8043823F00103C5F80438FEF778FD80
:102DD000370505D58E48FFF7BDFC8D48FEF75EFD33
:102DE000B0040CD5D5F8083813F0060FEB6823F4BF
:102DF00070530CBF43F4105343F4A053EB603107FE
:102E00001BD56368DB681BB9AB6923F00803AB61B2
:102E10002378052B0CD1D5F8003E7D489A071EBFBC
:102E2000D5F8003E23F00303C5F8003EFEF748FD49
:102E30006368DB680BB176489847F30274D4B70235
:102E400027D5D4F85490DFF8C8B100274FF0010A15
:102E500009EB4712D2F8003B03F44023B3F5802F6F
:102E600011D1D2F8003B002B0DDA62890AFA07F380
:102E700022EA0303638104EB8703DB68DB6813B199
:102E8000394658469847A36D01379B68FFB29F4269
:102E9000DED9F00617D5676D3A6AC2F30A1002F060
:102EA0000F0302F4F012B2F5802F00F08580B2F526
:102EB000402F08D104EB83030022DB681B6A07F56F
:102EC000805790426AD13003D5F8184813D5E103F2
:102ED00002D50020FFF744FEA20302D50120FFF730
:102EE0003FFE630302D50220FFF73AFE270302D517
:102EF0000320FFF735FE75037FF550AFE00702D5DD
:102F00000020FFF7C1FEA10702D50120FFF7BCFE9C
:102F1000620702D50220FFF7B7FE23077FF53EAF19
:102F20000320FFF7B1FE39E7636DDFF8E4A00193FA
:102F300000274FF00109A36D9B685FFA87FB9B4553
:102F40003FF67DAF019B03EB4B13D3F8001901F45F
:102F50004021B1F5802F1FD1D3F8001900291BDAC9
:102F6000D3F8001941F09041C3F80019D3F80019C3
:102F70000029FBDB5946606DFFF718FC218909FA2F
:102F80000BF321EA0303238104EB8B03DB689B68CB
:102F900013B15946504698470137CCE7910708BF0F
:102FA000D7F80080072A98BF03F8018B02F10102CD
:102FB00098BF4FEA182884E7023304EB830207F531
:102FC00080575268D2F818C0DCF80820DCE9001CF1
:102FD000A1EB0C0C002188420AD104EB8304636846
:102FE0009B699A6802449A605A6802445A606AE788
:102FF00011F0030F08BFD7F800808C4588BF02F896
:10300000018B01F1010188BF4FEA1828E3E700BFF7
:10301000F82F0020436D03EB4111D1F8003B43F43E
:103020000013C1F8003B7047436D03EB4111D1F829
:10303000003943F40013C1F800397047436D03EBC6
:103040004111D1F8003B23F40013C1F8003B704755
:10305000436D03EB4111D1F8003923F40013C1F89B
:103060000039704700F1604303F561430901C9B2BB
:1030700083F80013012200F01F039A4043099B00CC
:1030800003F1604303F56143C3F880211A60704780
:1030900030B5039C0172043304FB0325C0E90653D9
:1030A000049B03630021059BC160C0E90000C0E9E7
:1030B0000422C0E90842C0E90A11436330BD0000A0
:1030C000416A0022C0E90411C0E90A22C2606FF01F
:1030D0000101FEF7FFBE0000D0E90432934201D1A6
:1030E000C2680AB9181D704700207047036919604B
:1030F000C2680132C260C2691344826903619342AB
:1031000024BF436A03610021FEF7D8BE38B50446E8
:103110000D46E3683BB16269131D1268A362134454
:10312000E362002007E0237A33B929462046FEF700
:10313000B5FE0028EDDA38BD6FF00100FBE70000B6
:10314000C368C269013BC360436913448269436138
:10315000934224BF436A436100238362036B03B13C
:103160001847704770B53023044683F31188866A88
:103170003EB9FFF7CBFF054618B186F31188284604
:1031800070BDA36AE26A13F8015BA362934202D3A3
:103190002046FFF7D5FF002383F31188EFE70000F7
:1031A0002DE9F84F04460E46174698464FF0300971
:1031B00089F311880025AA46D4F828B0BBF1000F86
:1031C00009D141462046FFF7A1FF20B18BF31188BA
:1031D0002846BDE8F88FD4E90A12A7EB050B521A6E
:1031E000934528BF9346BBF1400F1BD9334601F1ED
:1031F000400251F8040B43F8040B9142F9D1A36A41
:1032000040334036A3624035D4E90A239A4202D3C0
:103210002046FFF795FF8AF31188BD42D8D289F383
:103220001188C9E730465A46FDF752FDA36A5B4450
:103230005E44A3625D44E7E710B5029C017204336B
:1032400003FB0421C0E906130023C0E90A33039BF2
:103250000363049BC460C0E90000C0E90422C0E924
:103260000842436310BD0000026AC260426AC0E9BE
:1032700004220022C0E90A226FF00101FEF72ABEF3
:10328000D0E904239A4201D1C26822B9184650F805
:10329000043B0B60704700231846FAE7C368C26915
:1032A0000133C3604369134482694361934224BF7D
:1032B000436A43610021FEF701BE000038B50446B1
:1032C0000D46E3683BB123691A1DA262E26913440B
:1032D000E362002007E0237A33B929462046FEF74F
:1032E000DDFD0028EDDA38BD6FF00100FBE70000DE
:1032F00003691960C268013AC260C26913448269F5
:103300000361934224BF436A036100238362036B1A
:1033100003B118477047000070B530230D460446CE
:10332000114683F31188866A2EB9FFF7C7FF10B1E3
:1033300086F3118870BDA36A1D70A36AE26A013327
:103340009342A36204D3E16920460439FFF7D0FF1A
:10335000002080F31188EDE72DE9F84F04460D4673
:10336000904699464FF0300A8AF311880026B346FA
:10337000A76A4FB949462046FFF7A0FF20B187F35F
:1033800011883046BDE8F88FD4E90A073A1AA8EB4D
:103390000607974228BF1746402F1BD905F1400367
:1033A00055F8042B40F8042B9D42F9D1A36A403311
:1033B000A3624036D4E90A239A4204D3E169204645
:1033C0000439FFF795FF8BF311884645D9D28AF36C
:1033D0001188CDE729463A46FDF77AFCA36A3B44BB
:1033E0003D44A3623E44E5E7D0E904239A4217D165
:1033F000C3689BB1836A8BB1043B9B1A0ED01360E8
:10340000C368013BC360C3691A44836902619A427D
:1034100024BF436A03610023836201231846704777
:103420000023FBE700F030B94FF08043586A704743
:103430004FF08043002258631A610222DA6070471D
:103440004FF080430022DA60704700004FF0804365
:1034500058637047FEE7000070B51B4B0163002501
:10346000044686B0586085620E4600F0BFF804F14D
:103470001003C4E904334FF0FF33C4E90635C4E94F
:103480000044A560E562FFF7CFFF2B460246C4E982
:10349000082304F134010D4A256580232046FEF7F8
:1034A000B3FC0123E0600A4A03750092726801923E
:1034B000B268CDE90223074B6846CDE90435FEF733
:1034C000CBFC06B070BD00BF90280020203D000856
:1034D000253D000855340008024AD36A1843D062DB
:1034E000704700BF282600204B6843608B688360CC
:1034F000CB68C3600B6943614B6903628B694362AC
:103500000B6803607047000008B5264B26481A690F
:1035100040F2FF110A431A611A6922F4FF7222F085
:1035200001021A611A691A6B0A431A631A6D0A4377
:103530001A651E4A1B6D1146FFF7D6FF02F11C01EA
:1035400000F58060FFF7D0FF02F1380100F58060E0
:10355000FFF7CAFF02F1540100F58060FFF7C4FFD6
:1035600002F1700100F58060FFF7BEFF02F18C01EF
:1035700000F58060FFF7B8FF02F1A80100F5806058
:10358000FFF7B2FF02F1C40100F58060FFF7ACFF66
:1035900002F1E00100F58060FFF7A6FFBDE80840FA
:1035A00000F0EEB800380240000002402C3D000858
:1035B00008B500F067FAFEF705FCFFF793F8BDE8E1
:1035C0000840FEF773BE000070470000EFF3098368
:1035D00005494A6B22F001024A63683383F3098884
:1035E000002383F31188704700EF00E0302080F360
:1035F000118862B60C4B0D4AD96821F4E0610904C8
:10360000090C0A43DA60D3F8FC20094942F08072C1
:10361000C3F8FC200A6842F001020A602022DA772F
:1036200083F82200704700BF00ED00E00003FA05B8
:10363000001000E010B5302383F311880E4B5B6857
:1036400013F4006314D0F1EE103AEFF30984683CF0
:103650004FF08073E361094BDB6B236684F30988C9
:10366000FEF790FB10B1064BA36110BD054BFBE7C5
:1036700083F31188F9E700BF00ED00E000EF00E000
:103680002F030008320300080F4B1A6C42F00102AE
:103690001A641A6E42F001021A660C4A1B6E936895
:1036A00043F0010393604FF0804353229A624FF03E
:1036B000FF32DA6200229A615A63DA605A600122AC
:1036C0005A611A60704700BF00380240002004E0D1
:1036D0004FF0804208B51169D3680B40D9B2C94395
:1036E0009B07116107D5302383F31188FEF780FB18
:1036F000002383F3118808BD1F4B1A696FEAC25279
:103700006FEAD2521A611A69C2F308021A614FF0C5
:10371000FF301A695A69586100215A6959615A691A
:103720001A6A62F080521A621A6A02F080521A62B1
:103730001A6A5A6A58625A6A59625A6A1A6C42F08C
:1037400080521A641A6E42F080521A661A6E0B4A40
:10375000106840F480701060186F00F44070B0F58D
:10376000007F1EBF4FF4803018671967536823F439
:103770000073536000F05EB90038024000700040F2
:10378000334B4FF080521A64324A4FF4404111607B
:103790001A6842F001021A601A689107FCD59A680B
:1037A00022F003029A602A4B9A6812F00C02FBD1B5
:1037B000196801F0F90119609A601A6842F48032C0
:1037C0001A601A689203FCD55A6F42F001025A67D8
:1037D0001F4B5A6F9007FCD51F4A5A601A6842F077
:1037E00080721A601B4A53685904FCD5184B1A683A
:1037F0009201FCD5194A9A60194B1A68194B9A42E2
:10380000194B21D1194A1168194A91421CD140F231
:1038100005121A60144A136803F00F03052BFAD13E
:103820000B4B9A6842F002029A609A6802F00C020E
:10383000082AFAD15A6C42F480425A645A6E42F411
:1038400080425A665B6E704740F20572E1E700BF46
:103850000038024000700040085440070094883847
:10386000002004E011640020003C024000ED00E074
:1038700041C20F41074A08B5536903F00103536180
:1038800023B1054A13680BB150689847BDE808405A
:10389000FFF7D0BE003C014070300020074A08B559
:1038A000536903F00203536123B1054A93680BB1D6
:1038B000D0689847BDE80840FFF7BCBE003C014017
:1038C00070300020074A08B5536903F004035361C0
:1038D00023B1054A13690BB150699847BDE8084008
:1038E000FFF7A8BE003C014070300020074A08B531
:1038F000536903F00803536123B1054A93690BB17F
:10390000D0699847BDE80840FFF794BE003C0140ED
:1039100070300020074A08B5536903F01003536163
:1039200023B1054A136A0BB1506A9847BDE80840B5
:10393000FFF780BE003C014070300020164B10B5F0
:103940005C6904F478725A61A30604D5134A936A39
:103950000BB1D06A9847600604D5104A136B0BB1BF
:10396000506B9847210604D50C4A936B0BB1D06B72
:103970009847E20504D5094A136C0BB1506C98477F
:10398000A30504D5054A936C0BB1D06C9847BDE8EC
:103990001040FFF74FBE00BF003C014070300020D8
:1039A000194B10B55C6904F47C425A61620504D578
:1039B000164A136D0BB1506D9847230504D5134A71
:1039C000936D0BB1D06D9847E00404D50F4A136E88
:1039D0000BB1506E9847A10404D50C4A936E0BB1FD
:1039E000D06E9847620404D5084A136F0BB1506F2C
:1039F0009847230404D5054A936F0BB1D06F9847BD
:103A0000BDE81040FFF716BE003C014070300020BA
:103A100008B50348FDF7C4FABDE80840FFF70ABE41
:103A2000BC23002008B5FFF753FEBDE80840FFF7B0
:103A300001BE0000062108B50846FFF713FB06216A
:103A40000720FFF70FFB06210820FFF70BFB0621DD
:103A50000920FFF707FB06210A20FFF703FB0621D9
:103A60001720FFF7FFFA06212820FFF7FBFA0721AE
:103A70001C20FFF7F7FABDE808400C212520FFF7CE
:103A8000F1BA000008B5FFF737FE00F00DF8FDF7BA
:103A90009BFCFDF781FEFDF759FDFFF795FDBDE8A5
:103AA0000840FFF7BFBC00000023054A1946013358
:103AB000102BC2E9001102F10802F8D1704700BFD3
:103AC00070300020034611F8012B03F8012B002A67
:103AD000F9D1704753544D3332463F3F3F00535462
:103AE0004D3332463430780053544D3332463432FD
:103AF000780053544D333246343436585800000061
:103B0000012033000010410001105A000310590039
:103B10000710310000000000D43A00081304000030
:103B2000DE3A000819040000E83A00082104000009
:103B3000F23A0008009600000000000000000000BB
:103B400000000000000000000000000089130008D1
:103B500075130008B11300089D130008A91300088D
:103B600095130008811300086D130008BD130008A9
:103B700000000000C9140008B5140008F114000882
:103B8000DD140008E9140008D5140008C114000869
:103B9000AD140008FD140008000000000100000042
:103BA0000000000063300000A43B000880260020D5
:103BB0009028002043534B590025424F4152442541
:103BC0002D424C002553455249414C250000000030
:103BD0000200000000000000E51600085117000870
:103BE00040004000302D0020402D00200200000049
:103BF000000000000300000000000000951700080E
:103C00000000000010000000502D00200000000007
:103C10000100000000000000F82F00200101020058
:103C20004922000859210008F5210008D92100087F
:103C300043000000383C000809024300020100C0B4
:103C400032090400000102020100052400100105F0
:103C50002401000104240202052406000107058254
:103C6000030800FF09040100020A00000007050123
:103C70000240000007058102400000001200000021
:103C8000843C000812011001020000400912415753
:103C900000020102030100000403090425424F4110
:103CA0005244250043534B593430350030313233C0
:103CB0003435363738394142434445460000000028
:103CC00000400000004000000040000000400000F4
:103CD00000000100000002000000020000000200DD
:103CE00000000200000002000000020000000200CC
:103CF00000000000D9180008911B00083D1C0008B6
:103D000040004000583000205830002001000000E2
:103D10006830002080000000400100000300000027
:103D20006D61696E0069646C650000000001A81691
:103D300000000000AAAAAAAA00011400FF9F000028
:103D40000000000070A70A00000000010000000051
:103D5000AAAAAAAA00000001FFFF000000000000BC
:103D6000000000000400001400000000AAAAAAAA93
:103D700004000014FFFF000000000000000000002D
:103D80000000000000000000AAAAAAAA000000008B
:103D9000FFFF000000000000000000000000000025
:103DA00000000000AAAAAAAA00000000FFFF00006D
:103DB0000000000000000000000000000000000003
:103DC000AAAAAAAA00000000FFFF0000000000004D
:103DD000000000000000000000000000AAAAAAAA3B
:103DE00000000000FFFF00000000000000000000D5
:103DF00000000000000000000A00000000000000B9
:103E000003000000000000000000000000000000AF
:103E100000000000000000000000000000000000A2
:103E20000000000000000000860400000000000008
:103E300000400F0000000000FF0000009828002054
:103E4000BC2300200096000000000800960000003F
:103E50000008000004000000983C0008000000007A
:103E60000000000000000000000000000000000052
:043E7000000000004E
:00000001FF
